:020000040800F2
:1000000000400020953700085D0400085F040008E8
:1000100000000000000000000000000000000000E0
:100020000000000000000000000000006104000863
:1000300000000000000000006304000865040008E0
:10004000E5370008E5370008E5370008E537000820
:10005000E5370008E5370008E5370008E537000810
:10006000E53700086D040008E5370008E5370008AB
:10007000E5370008E5370008E5370008E5370008F0
:10008000E5370008E5370008E5370008E5370008E0
:10009000E5370008E5370008E5370008E5370008D0
:1000A000E5370008E5370008E5370008E5370008C0
:1000B000E5370008E5370008E53700087D0400084B
:1000C00010B5064C2378002B07D1054B002B02D02E
:1000D000044800E000BF0123237010BD0801002088
:1000E0000000000040380008044B10B5002B03D07E
:1000F0000349044800E000BF10BDC04600000000F6
:100100000C01002040380008002243088B4274D3C1
:1001100003098B425FD3030A8B4244D3030B8B4208
:1001200028D3030C8B420DD3FF22090212BA030C11
:100130008B4202D31212090265D0030B8B4219D3F2
:1001400000E0090AC30B8B4201D3CB03C01A524112
:10015000830B8B4201D38B03C01A5241430B8B425A
:1001600001D34B03C01A5241030B8B4201D30B0343
:10017000C01A5241C30A8B4201D3CB02C01A52416A
:10018000830A8B4201D38B02C01A5241430A8B422D
:1001900001D34B02C01A5241030A8B4201D30B0216
:1001A000C01A5241CDD2C3098B4201D3CB01C01A30
:1001B000524183098B4201D38B01C01A524143093A
:1001C0008B4201D34B01C01A524103098B4201D328
:1001D0000B01C01A5241C3088B4201D3CB00C01A95
:1001E000524183088B4201D38B00C01A524143080D
:1001F0008B4201D34B00C01A5241411A00D2014632
:10020000524110467047FFE701B5002000F006F8A4
:1002100002BDC0460029F7D076E770477047C04658
:1002200030B589B01422002103A803F001FB134B61
:1002300059698020C002014359615A690240019204
:10024000019A5A69802189020A435A615B690B400D
:100250000293029B8025AD01094C00222900200059
:1002600001F0CAFD0395012304930023059306932F
:1002700003A9200001F0F4FC09B030BD00100240D9
:100280000004004800B583B0094A516901231943AD
:100290005161526913400193019B00220021092002
:1002A00001F092FE092001F0C1FE03B000BDC0467E
:1002B00000100240F0B585B00C22002101A803F027
:1002C000B7FA294C294B236000256560A560E560DD
:1002D000012626610827676125766576A676E5768C
:1002E000C223FF33E36125629E3BFF3BE654A662D7
:1002F000200000F01DFE019580235B01029306356E
:10030000039501A9200000F073FF019601A92000C8
:1003100000F06EFF0223019301A9200000F068FFA6
:100320000323019301A9200000F062FF042301933D
:1003300001A9200000F05CFF0523019301A9200022
:1003400000F056FF019501A9200000F051FF07239E
:10035000019301A9200000F04BFF019701A92000A3
:1003600000F046FF05B0F0BDFC0300200024014072
:1003700010B598B0302200210CA803F059FA1022D1
:10038000002107A803F054FA1C220021684603F05C
:100390004FFA30230B932F3B139310930F3311938A
:1003A0000BA800F0CBFF07230793043B089300241E
:1003B00009940A94012107A801F0AAFA80239B025C
:1003C00000930694684601F043FB18B010BD00008E
:1003D00070B501F011FCFFF7CBFFFFF721FFFFF72E
:1003E00051FFFFF767FF02F0E1FA08220C490D48C0
:1003F00000F05CFE8026B6010B4D01223100280082
:1004000001F0FAFCFA24A400200001F017FC0022FD
:100410003100280001F0F0FC200001F00FFCE9E7BA
:10042000EC030020FC0300200004004870B5802588
:10043000AD01094C01222900200001F0DDFC6420FF
:1004400001F0FCFB00222900200001F0D5FC642013
:1004500001F0F4FBEBE7C046000400487047FEE7FC
:100460007047704710B501F0D7FB10BD10B50248BA
:1004700001F055FD10BDC0463401002010B5024802
:1004800002F016F910BDC0467801002082B00A4B78
:10049000996901221143996199690A400092009A71
:1004A000DA69802149050A43DA61DB690B4001936F
:1004B000019B02B07047C0460010024030B589B0C1
:1004C00004001422002103A803F0B2F9274B22688C
:1004D0009A4201D009B030BD254B99698020800037
:1004E000014399619A6902400092009A59698020FB
:1004F0008002014359615A6902400192019A5A6986
:100500008021C9020A435A615B690B400293029B36
:10051000FF23039303250495902003A9C00501F050
:100520009FFB0123039304950025059503A911481A
:1005300001F096FB1048114B0360456085608023F5
:10054000C360803303618023DB0043612023836128
:1005500080235B01C36101F07FFC002803D1064BBF
:1005600023635C62B6E7FFF761FFF8E70024014010
:10057000001002400004004834010020080002403E
:100580004022835A02490B439BB28352002070479A
:1005900080BFFFFF4022835A02490B408352002054
:1005A0007047C0467F40000084B010B503910492AC
:1005B0000593402201238352002383520432835245
:1005C0000C328352FFF7DCFF002010BC08BC04B0E3
:1005D00018470000F0B50D78AD0045192B88B14AD9
:1005E0001340CA78012A54D0002A48D0022A03D0E6
:1005F000032A49D0012400E00024AB4A13439BB2F4
:100600002B800B789E00861935882DB2A74F3D4070
:100610002B439BB21A4392B232800B7B002B00D04B
:1006200094E04B78002B44D05023C25A82180B78A8
:10063000DB009B188022D20094466344CA8852088B
:1006400052001A800B789B00C3181A88520606D5F0
:100650001A883D001540964A2A4392B21A80CB78F8
:10066000012B1BD00B789B00C0180388914A1340C4
:1006700020225A408C4B13439BB2038051E08022CE
:10068000920013430024B8E7C022D2001343002491
:10069000B3E78022D20013430024AEE70B789B001F
:1006A000C0180388834A1A407F4B13439BB20380D0
:1006B00037E05025425B82180B78DB009B187E4A9E
:1006C00094466344CA88520852001A80425B8218DA
:1006D0000B78DB009B18794A944663440A69002A28
:1006E00021D11A88764D1540764A2A431A800B7814
:1006F0009B00C3181A88520406D51A886B4D154002
:10070000714A2A4392B21A800B789B00C018028863
:100710006E4B1A40C0239B015A40634B13439BB25C
:1007200003802000F0BD3E2A06D85508D20700D528
:100730000135AD021D80DAE75509D20600D1013D31
:10074000AD02ADB25F4A15431D80D0E70B789B0028
:10075000C3181A88554D15405D4A2A4392B21A8033
:100760005025425B82180B78DB009B188022D20058
:10077000944663440A89520852001A80425B8218E8
:100780000B78DB009B184C4A944663444A89520814
:1007900052001A804B78002B3AD10B789B00C3187B
:1007A0001A88520406D51A88404D1540464A2A43F5
:1007B00092B21A800B789B00C3181A88520606D58D
:1007C0001A883A4D15403A4A2A4392B21A800B7859
:1007D0009B00C3181A88354D1540354A2A4392B2FA
:1007E0001A800A78920082181388384D1D40C02361
:1007F0009B016B402C4D2B439BB213800B789B00CD
:10080000C01803882B4A13402B439BB2038088E710
:100810000B789B00C3181A88520406D51A88234DFA
:100820001540294A2A4392B21A800B789B00C318BC
:100830001A88520606D51A881C4D15401C4A2A43B0
:1008400092B21A800B789B00C3181A88174D154076
:100850001D4A2A4392B21A80CB78012B16D00B780E
:100860009B00C3181A88134D2A40202555400E4A74
:100870002A4392B21A800B789B00C3181A88134936
:100880001140094A0A4392B21A804AE70B789B004A
:10089000C3181A88074D1540034A2A4392B21A809A
:1008A000E9E7C0468F89FFFF8080FFFF8F8FFFFF42
:1008B000C080FFFFBF8FFFFF04040000060400009C
:1008C000FF83FFFF0080FFFF80C0FFFF8FBFFFFFA0
:1008D0008081FFFF10B50B7B002B33D14B78002BB1
:1008E00018D00B789B00C3181A88520606D51A88B0
:1008F0004E4C14404E4A224392B21A800B789B0011
:10090000C01803884B4A1A404B4B13439BB20380D9
:10091000002010BD0B789B00C3181A88520406D51E
:100920001A88424C1440454A224392B21A800B78EE
:100930009B00C0180388424A1A403F4B13439BB2A6
:100940000380E5E74B78002B37D10B789B00C31869
:100950001A88520406D51A88344C1440374A224368
:1009600092B21A800B789B00C3181A88520606D5DB
:100970001A882E4C14402E4A224392B21A800B78C9
:100980009B00C3181A88294C1440294A224392B26A
:100990001A800C78A40004192388294A1340264A97
:1009A00013439BB223800B789B00C0180388214916
:1009B0000B401A4392B20280AAE70B789B00C3183F
:1009C0001A88520406D51A88184C14401B4A224330
:1009D00092B21A800B789B00C3181A88520606D56B
:1009E0001A88124C1440124A224392B21A800B7891
:1009F0009B00C3181A880D4C1440104A224392B22F
:100A00001A800C78A400041923880A4A13400A4A61
:100A100013439BB223800B789B00C01803880849BE
:100A20000B401A4392B2028072E7C0468F8FFFFFDD
:100A3000C080FFFFBF8FFFFF8080FFFF80C0FFFFF0
:100A40008FBFFFFF4B78002B0ED10B789B00C01897
:100A500002880C4B1A4080235B015A400A4B134317
:100A60009BB20380002070470B789B00C01803885E
:100A7000064A134010225A40034B13439BB2038093
:100A8000F0E7C0468FBFFFFF8080FFFFBF8FFFFFF3
:100A900010B50B7B002B39D14B78002B1CD00B7879
:100AA0009B00C3181A88520606D51A88184C1440A1
:100AB000184A224392B21A80CB78012B26D00B78A9
:100AC0009B00C0180388144A134020225A40134B3D
:100AD00013439BB2038019E00B789B00C3181A885C
:100AE000520406D51A880A4C14400D4A224392B289
:100AF0001A800B789B00C01802880A4B1A40C0234A
:100B00009B015A40054B13439BB20380002010BD4C
:100B10008F8FFFFFC080FFFFBF8FFFFF8080FFFF31
:100B200080C0FFFF8FBFFFFF002902D14C2380222E
:100B3000C2520020704700005822835A02490B43DA
:100B40009BB28352002070470080FFFF4423C05AAD
:100B500080B270470020704710B501335B0812184F
:100B60008020C0008446624407E008784C78240264
:100B70000443148002320231013B002BF5D110BD39
:100B800070B505000C00497801292BD0A2692369B2
:100B90009A4200D8D8E0D21AA261227B002A00D063
:100BA000E9E05032A95A69182278D2005218A049B7
:100BB0008C466244002B00D0CAE013889D4919403E
:100BC0009D4B0B43138023789B00ED182A889B4B89
:100BD0001A40C0239B015A40994B13439BB22B8070
:100BE000002070BDA26923699A421DD9D21AA26160
:100BF000227B002A1CD0227890002818008840060A
:100C000064D5002939D15031695A6918D200521877
:100C100087498C466244002B1CD1118885480840C6
:100C200085490143118031E00023A3611300DFE710
:100C30009EB2E288330061692800FFF78DFF5023E0
:100C4000EA5AAA182378DB009B187E4A944663442C
:100C50001E802EE03E2B06D85908D80700D501315A
:100C60008902118012E05909D80600D101398902A0
:100C700089B271480143118008E05021695A69180E
:100C8000D20052186A498C466244138062899BB232
:100C900061692800FFF760FF6378002B47D1237854
:100CA0009B00EB181A8868491140684A0A4392B2BF
:100CB0001A8023789B00ED182B88654A1340302258
:100CC0005A405F4B13439BB22B8089E7002923D105
:100CD0005031695A6918D20052185A498C466244F8
:100CE000002B06D111885348084053490143118015
:100CF0001BE03E2B06D85908D80700D501318902E0
:100D0000118012E05909D80600D10139890289B24F
:100D100049480143118008E05021695A6918D200FE
:100D2000521848498C46624413802289AFE7012B50
:100D3000BFD123789B00EB181A8843491140454ADC
:100D40000A4392B21A80B4E70023A361130024E798
:100D50003E2B06D85908DB0700D5013189021180E6
:100D600031E75909DB0600D10139890289B2324BDA
:100D70001943118027E7002910D15022A95A691878
:100D80002278D20052182F498C466244002B1AD187
:100D90001188284808402849014311806278002AB8
:100DA00037D15032A95A69182278D20052182049F6
:100DB0008C466244002B19D113881E4919401E4BE2
:100DC0000B431380FFE63E2B06D85908D80700D501
:100DD000013189021180E1E75909D80600D10139B2
:100DE000890289B2144801431180D7E73E2B06D807
:100DF0005908DB0700D5013189021180E3E6590962
:100E0000DB0600D10139890289B20B4B19431180ED
:100E1000D9E6012A00D0D6E64F32A95A69182278BD
:100E2000D200521802498C4662441380CBE6C04679
:100E300006040000FF83FFFF0080FFFF8FBFFFFF5E
:100E40008080FFFF020400008F8FFFFFC080FFFF44
:100E5000BF8FFFFF80C0FFFF30B55D0812188020F4
:100E6000C0008446624407E01488A4B202320C70C9
:100E7000240A4C700231013D002DF5D1DB0701D56C
:100E800013880B7030BD000030B583B00400002320
:100E900001930368996803220A40012A0ED09968D9
:100EA000204A114212D19A6801210A439A601E4BCE
:100EB00018681E49FFF728F9019015E01A68D20753
:100EC0002DD4DA681204EAD5002008E0A36B1022C2
:100ED0001343A363E36B0F3A1343E363012003B0AF
:100EE00030BD019B013B0193019B002BF9D100F028
:100EF0009FFE050023681B68DB070ED400F098FEF8
:100F0000401B0228F6D9A36B10221343A363E36BA3
:100F10000F3A1343E3630120E1E70020DFE70020FD
:100F2000DDE7C046170000800401002040420F00AA
:100F300070B5041E00D1B1E0836B002B7ED0A36B93
:100F4000DB0600D5A4E021688B6804221A4000D09B
:100F50009EE0A36B524803400630FF300343A36377
:100F6000886803230340012B6ED0CB68182083438D
:100F7000A0680343CB6021680B699B009B086068F5
:100F800003430B612168CB6846480340CB60237E56
:100F90009B03617EC9030B43A17E48030343A06A00
:100FA000012858D0802040010343E06803432069B2
:100FB000022852D013432422A25C52001343E27E43
:100FC000012A4CD0E269C221FF318A4202D0216A53
:100FD0000A4313432168CA681A43CA60E26A80213F
:100FE00049058A420DD0012A0BD0022A09D0032AD2
:100FF00007D0042A05D0052A03D0062A01D0072AE3
:101000000AD1206841690722914341612068416902
:10101000E56A2A400A4342612268D26822490A40AE
:101020009A422BD0A36B12229343023A1343A36339
:10103000E36B0F3A1343E36301202EE0C3633422D2
:101040008354FFF73BFA7AE70B68DB079AD4CB6847
:101050001B0497D489E71000A6E70422AAE7002919
:1010600003D1802252021343ACE7A26B20210A4332
:10107000A263E26B1F390A43E263A3E70023E36341
:10108000A36B03229343023A1343A363002004E0BB
:10109000A36B10221343A363012070BD0120FCE762
:1010A000FDFEFFFF1902FEFFE7FF3F83F8B50400D6
:1010B0000E00170003689B685B073ED43423C35CB3
:1010C000012B3CD034230122C254437E012B32D069
:1010D000FFF7DAFE051E2CD1A36B1A4A1A408023B3
:1010E0005B001343A3630023E3633422A354236B05
:1010F000154A9A62236B154ADA62236B144A1A6303
:1011000023681C221A602268536810210B43536025
:101110002268D3680F390B43D360216840313B000C
:101120003200206B00F0C0FE2268936804210B435C
:1011300093602800F8BD0025CEE70225F9E70225D7
:10114000F7E7C046FEF0FFFF59110008CB11000879
:10115000D71100087047000010B5436A9A6B502100
:10116000114203D01B6B1B6B984710BD996B8022FB
:1011700092000A439A631A68D068C02109010842A4
:1011800013D1997E002910D1116809070DD59168F6
:1011900049070ED451680C20814351609A6B09496C
:1011A0000A400431FF310A439A631800FFF7D2FF67
:1011B000DBE79A6B20210A439A63DA6B1F390A43F3
:1011C000DA63F2E7FEFEFFFF704710B5406AFFF7F3
:1011D000FBFF10BD704710B5406A836B402213437C
:1011E0008363C36B3C3A1343C363FFF7F3FF10BD44
:1011F00030B583B00400002301933433C35C012B6A
:1012000000D18AE034230122C25403689A6852074D
:1012100075D4434A4868904256D09A6A01200D68B6
:10122000A84002439A62E36A8022520593421ED08C
:10123000012B1CD0022B1AD0032B18D0042B16D054
:10124000052B14D0062B12D0072B10D02268506922
:10125000072303408868984209D0506907239843C0
:101260005061206842698D682B40134343610B68CD
:101270001A00103A022A4CD82A4A1268102B0ED0B3
:10128000112B09D080235B041343264A13600B689B
:10129000102B07D0002037E08023DB03F4E7802306
:1012A0001B04F1E7204B18682049FEF72DFF83004F
:1012B00018184300019302E0019B013B0193019B3D
:1012C000002BF9D100201FE09A6A01200D68A84088
:1012D00082439A620B681A00103A022A1BD8114AFC
:1012E0001268102B09D0112B05D0114B13400D4A59
:1012F0001360002008E00F4BF8E70F4BF6E7836B15
:10130000202213438363012034230022E25403B0DC
:1013100030BD0020F8E70020F6E70220F7E7C046DE
:1013200001100000082701400401002040420F0086
:10133000FFFFFFFEFFFFBFFFFFFF7FFF70B582B023
:10134000041E00D185E20368DB072BD5B34B5A6836
:101350000C231340042B1DD0B04B5A680C231340B0
:10136000082B0ED06368012B41D0002B56D1AB4B1C
:101370001A68AB490A401A601A68AA490A401A60FA
:101380003BE0A64B5B68C02252021340802252020F
:101390009342E7D1A14B1B689B0303D56368002BE5
:1013A00000D159E223689B0778D59C4B5B680C22DF
:1013B0001A4262D0994B5A680C231340082B53D021
:1013C000E368002B00D18BE0944A136801210B43A2
:1013D000136000F02DFC0500904B1B689B0776D432
:1013E00000F026FC401B0228F6D9032032E28B4A8B
:1013F000116880235B020B4313606368002B25D0C8
:1014000000F016FC0500854B1B689B03CAD400F056
:101410000FFC401B6428F6D903201BE2052B09D0E2
:101420007E4B1A687E490A401A601A687D490A4054
:101430001A60E2E7794B19688022D2020A431A60E7
:101440001968802252020A431A60D6E700F0F0FBC6
:101450000500724B1B689B03A4D500F0E9FB401B01
:101460006428F6D90320F5E16C4B5B68C022520278
:101470001340802212029342A2D1684B1B689B0743
:1014800004D5E368012B01D00120E3E163490B6837
:10149000F82293432269D20013430B6023681B0791
:1014A00044D5E369002B2ED05C4A536A01210B43DB
:1014B000536200F0BDFB0500584B5B6A9B0735D4B7
:1014C00000F0B6FB401B0228F6D90320C2E15349C5
:1014D0000B68F82293432269D20013430B60DDE7C7
:1014E0004E4A136801218B43136000F0A1FB0500F5
:1014F0004A4B1B689B07D1D500F09AFB401B022882
:10150000F6D90320A6E1454A536A01218B43536271
:1015100000F08EFB0500414B5B6A9B0706D500F08F
:1015200087FB401B0228F6D9032093E123685B0761
:1015300000D47FE0394BDB69DB001DD4374AD16929
:10154000802040050143D161D36903400193019B91
:101550000125354B1B68DB0510D5A368012B21D075
:10156000002B36D12D4B1A6A01218A431A621A6A5E
:1015700003318A431A621AE00025EAE72A4A116811
:1015800080235B000B43136000F052FB0600264BE8
:101590001B68DB05E1D400F04BFB801B6428F6D907
:1015A000032057E11D4A136A01210B431362A3680C
:1015B000002B24D000F03CFB0600184B1B6A9B0755
:1015C00036D400F035FB801B184B9842F5D9032028
:1015D00040E1052B09D0114B1A6A01218A431A6296
:1015E0001A6A03318A431A62E1E70C4B1A6A042132
:1015F0000A431A621A6A03390A431A62D7E700F0EB
:1016000017FB0600054B1B6A9B0711D500F010FB6A
:10161000801B064B9842F5D903201BE100100240C5
:10162000FFFFFEFFFFFFFBFF00700040881300007C
:10163000012D3AD02368DB0610D56369012B3AD01F
:10164000053358D1884A536B04218B435363536B42
:10165000F4318B43A169C9000B43536323689B0694
:1016600000D482E0804B5A680C2313400C2B60D0CE
:101670007D4B5A680C231340082B53D0236A002B50
:1016800060D0794A516B80235B020B43536300F0B7
:10169000CFFA0500744B5B6BDB0366D400F0C8FA2D
:1016A000401B0228F6D90320D4E06F4AD3696F4962
:1016B0000B40D361BEE76C4B5A6B04210A435A635B
:1016C0005A6B03390A435A6300F0B2FA0500664BBD
:1016D0005B6B9B0706D400F0ABFA401B0228F6D9DF
:1016E0000320B7E060494B6BF8229343A269D20014
:1016F00013434B63B2E75C4B5A6B04210A435A63B2
:101700005A6B03398A435A6300F092FA0500564B2C
:101710005B6B9B07A2D500F08BFA401B0228F6D921
:10172000032097E0504B5B68C02252021340934263
:10173000A4D14D4B5B6BDB0317D5236A012B14D06F
:10174000012087E0484A536B49490B40536300F03E
:101750006FFA0500444B5B6BDB0306D500F068FABB
:10176000401B0228F6D9032074E0636A002B00D1E5
:1017700074E03D4A51680C220A40082A4DD0022BE1
:1017800012D0394A13683B490B40136000F050FAFD
:101790000400354B1B689B013DD500F049FA001B46
:1017A0000228F6D9032055E02F4A136831490B402F
:1017B000136000F03DFA05002B4B1B689B0106D51A
:1017C00000F036FA401B0228F6D9032042E0264BEF
:1017D000DA6A0F218A43216B0A43DA625A68264982
:1017E0000A40E16AA06A01430A435A6019688022EC
:1017F00052040A431A6000F01BFA04001A4B1B68DB
:101800009B0106D400F014FA001B0228F6D903202D
:1018100020E000201EE000201CE0012B20D0124B15
:101820005A68D96AC0235B021340A06A834201D080
:1018300001200FE00F230B40216B8B4201D00120D0
:1018400008E0F0239B031A40E36A9A420AD0012081
:1018500000E0012002B070BD0120FBE70020F9E7A5
:101860000120F7E70020F5E700100240FFFFFFEF3F
:10187000FFFFFEFFFFFFFFFEFF7FC2FF30B589B015
:1018800004AA1F4B180032C832C2110002680A6055
:101890006A46103313CB13C21B681360194B5A6886
:1018A0000C231340082B04D00C2B26D0164809B06B
:1018B00030BD910C0F23194004A8445C1149C96A3A
:1018C0000B406946C95CC0235B021A4080235B025F
:1018D0009A4208D0C0235B029A4209D00A48FEF718
:1018E00013FC6043E3E70848FEF70EFC6043DEE7C5
:1018F0000648FEF709FC6043D9E70448D7E7C0462D
:10190000583800080010024000127A00006CDC0217
:1019100070B504000D00002800D189E0464B1A681C
:10192000012313408B420BD243490B68012293439E
:101930002B430B600B681A40AA4201D0012078E0CB
:1019400023689A070ED55B0705D53C4A5168E0230A
:10195000DB000B435360394A5368F0218B43A16885
:101960000B4353602368DB0735D56368012B09D02F
:10197000022B24D0032B28D0304A1268920705D4BA
:10198000012056E02D4A1268920353D52B494A682C
:101990000320824313434B6000F04AF90600274BB3
:1019A0005B680C221A4063689B009A4213D000F0D7
:1019B0003FF9801B224B9842F1D9032039E01F4A9E
:1019C00012689201E2D4012033E01C4A526BD20328
:1019D000DCD401202DE0184B1A6801231340AB42E0
:1019E0000BD915490B68012293432B430B600B68FD
:1019F0001A40AA4201D001201BE023685B0706D5EC
:101A00000E4A53680F490B40E1680B435360FFF7E0
:101A100035FF0A4B5A6812090F2313400A4AD35C58
:101A2000D8400A4B1860002000F0BEF8002000E00B
:101A3000012070BD0120FCE70020024000100240A0
:101A400088130000FFF8FFFF64390008040100203C
:101A500070B582B004000368DB0335D54B4BDB69FE
:101A6000DB0066D4494AD169802040050143D16139
:101A7000D36903400193019B0125454B1B68DB059E
:101A800059D5424B1B6AC0229200134013D06168A3
:101A90000A409A420FD03D4B186A3E4A02401E6AE5
:101AA0008021490231431962196A3B4E3140196263
:101AB0001A62C30753D4354A136A36490B4061682A
:101AC0000B431362012D59D02368DB0706D52F4A3B
:101AD000136B03218B43A1680B43136323689B079C
:101AE00006D52A4A136B2D490B40E1680B4313635B
:101AF00023689B0606D5254A136B10218B43216969
:101B00000B43136323689B0306D5204A136B802184
:101B10008B43A1690B43136323685B0533D51B4AD1
:101B2000136B40218B4361690B431363002002B0A8
:101B300070BD0025A1E7164A116880235B000B43A6
:101B4000136000F075F80600114B1B68DB0598D494
:101B500000F06EF8801B6428F6D90320E7E700F058
:101B600067F80600094B1B6A9B07A4D400F060F8D5
:101B7000801B0B4B9842F5D90320D8E7D36909495C
:101B80000B40D361A0E70020D1E7C046001002401F
:101B900000700040FFFCFFFFFFFFFEFFFFFFFCFFA8
:101BA00088130000FFFFFFEF10B504000F4B1978FA
:101BB000FA208000FEF7A8FA01000D4B1868FEF726
:101BC000A3FA00F03FFA00280DD1032C01D901201F
:101BD0000AE0013000222100404200F0F5F9054BF7
:101BE0001C60002000E0012010BDC0460000002065
:101BF000040100200400002010B5064A13681021DB
:101C00000B4313600020FFF7CFFFFEF73FFC0020DF
:101C100010BDC04600200240034A1168034B1B78E8
:101C20005B1813607047C0463C0400200000002091
:101C3000014B18687047C0463C04002070B5040092
:101C4000FFF7F6FF0500631C02D0044B1B78E41875
:101C5000FFF7EEFF401BA042FAD370BD000000204A
:101C6000F0B5C64600B582B0002338E0042600E097
:101C70000026AE4035003D430234A400574EA55126
:101C8000574C25684246D4432E0026404A68D2036A
:101C900002D5424615432E00514D2E606D682E0030
:101CA00026404A68920302D5424615432E004C4D09
:101CB0006E60AD682E0026404A68D20202D54246C8
:101CC00015432E00464DAE60ED682C404A689202E6
:101CD00002D542462A431400414AD46001330A68BF
:101CE0001400DC4076D001259D402A409046F5D076
:101CF0004C68022C01D0122C0ED1DC080834A40050
:101D0000275807261E40B6000F22B24097430A69A3
:101D1000B24016003E43265002685F0003242600AE
:101D2000BE40F643324094464A681440BC40624686
:101D3000144304604C68621E012A03D9112C01D09F
:101D4000122C10D184683440A446CC68BC40624652
:101D5000144384604468AC434A6812090125154065
:101D60009D4025434560C46826408C68BC40344390
:101D7000C4604A68D200B1D51A4DAE690124264329
:101D8000AE61AD692C400194019C9C08A51CAD007E
:101D9000124EAF5903261E40B5000F26AE40B74382
:101DA0009026F605B04200D162E70F4EB0420BD04C
:101DB0000E4EB0420AD00E4EB04209D00D4EB04287
:101DC00000D153E7052654E7012652E7022650E7E3
:101DD00003264EE702B004BC9046F0BD000001406F
:101DE00000040140001002400004004800080048C0
:101DF000000C004800100048002A01D181627047A1
:101E00008161FCE770B5C56B0124066CB4406C6061
:101E1000046863604368102B04D00368996003680A
:101E2000DA6070BD03689A600368D960F9E7000062
:101E300010B504000368064A944663441800142150
:101E4000FEF762F980002064024BE36310BDC046D8
:101E5000F8FFFDBF0000024070B5041E20D0212510
:101E60000223435501680B680E4A1A404368806894
:101E70000343E06803432069034360690343A069A7
:101E80000343E069034313430B602000FFF7D0FFD7
:101E90000023A363012262551F32A354002070BDAA
:101EA0000120FCE70FC0FFFF70B504002020205C7C
:101EB000012832D02020012525540130205C012842
:101EC00004D020230022E254022070BD20300135CE
:101ED00025540020A063256828680126B0432860A7
:101EE0002000FFF78FFFE36A002B0BD022681368F6
:101EF0000E210B4313602268136801210B4313600A
:101F00000020E2E7226813680A210B43136022686D
:101F1000136806398B431360EDE70220D5E770B5EF
:101F2000C36B1A6804682568016C04238B401A424D
:101F300012D06B0710D523689B0603D423680422B4
:101F400093432360C26B0423016C8B405360C36ACC
:101F5000002B00D0984770BD02238B401A4218D046
:101F6000AB0716D523689B0606D423680A22934341
:101F700023602123093AC254C26B0223016C8B40B7
:101F8000536020230022C254836A002BE3D0984779
:101F9000E1E708238B401A42DDD02B07DBD523680D
:101FA0000E2293432360C26B01231900046CA140ED
:101FB00051608363212283541F330022C254036B78
:101FC000002BC8D09847C6E770B5002811DB8308FE
:101FD000144DC0339B005C5903221040C000FC32FA
:101FE00016008640B44389010A40824022435A5178
:101FF00070BDC0B20F230340083B9B0806339B0013
:10200000094A944663445D6803242040C000FF22CF
:1020100014008440A543890111408140294359603F
:10202000E6E7C04600E100E000ED00E0002805DB47
:102030001F2318401E3B8340014A13607047C0466F
:1020400000E100E001380A4B98420FD8094A50607D
:102050000948036A1B021B0AC02109060B430362DD
:102060000023936007331360002070470120FCE7D2
:10207000FFFFFF0010E000E000ED00E030B587B0AA
:10208000041E61D0314BC35C002B07D02F4B0322C1
:10209000E2542068FEF77EFA00231AE08A239B00B0
:1020A0000022C25400F09EFCF0E75A01A218110071
:1020B00029310120087001390B70D38610002B30B4
:1020C000002101709163D1639A1C520111510133B7
:1020D000DBB260688342E8D3002215E05301E318C5
:1020E0001D002A35FF3500212970013D2A70033576
:1020F00029700D3529603D33FF33196013000A3311
:102100005B0119510132D2B29042E7D86A462300EE
:10211000103323CB23C203CB03C26168A268E368F8
:102120002068FEF741FA24230022E254074B0132D3
:10213000E254E369012B02D0002007B030BD20003B
:1021400000F01FFC0020F8E70120F6E7290200005C
:1021500070B504008A239B00C35C012B0DD08A2537
:10216000AD00012343550068FEF7E6FC2068FEF74A
:1021700007FA00236355002070BD0220FCE770B50C
:1021800004008A239B00C35C012B0CD08A25AD0080
:10219000012343552333C1540068FEF7C5FC0023D7
:1021A0006355002070BD0220FCE770B5050048B201
:1021B000002827DB07240C40640120002930FF3071
:1021C00028182C192A34FF340026267007242140B1
:1021D00001700261C3704278002A00D0C181022BD5
:1021E0001BD08A239B00EB5C012B19D08A24A4000E
:1021F00001232B5501002868FEF7ECF900232B552D
:10220000002070BD07240C406401200028302818ED
:102210002C19293401262670D8E700230371E0E742
:102220000220EEE770B504004BB2002B1FDB072342
:102230000B405B011A002932FF328218C3182A337F
:10224000FF33002018700723194011708A239B0068
:10225000E35C012B16D08A25AD00012363551100E4
:102260002068FEF737FB00236355002070BD07236D
:102270000B405B011A0028328218C3182933012051
:102280001870E0E70220F1E770B507250D406C01FA
:1022900021002931FF314118041926003D36FF364F
:1022A00032602A000A325201135082180023536010
:1022B00022002A32FF3213702934FF342570002D9A
:1022C00004D00068FEF75CFC002070BD0068FEF7DB
:1022D00057FCF9E770B507250D406C012100283146
:1022E00041180419E263AA1C5201135082180023FA
:1022F00053602300293301221A7028342570002DE1
:1023000004D00068FEF73CFC002070BD0068FEF7BA
:1023100037FCF9E7F0B5C64600B505002868442348
:10232000C35A1BB2002B00DBAAE14423C35A9BB261
:102330000F241C4000D0BCE0DB0651D503889BB2C3
:102340001A0500D57FE01BB2002BE7DA0388CE4ADE
:10235000134080221343038028685023C35A9422D9
:102360005200AA5CD2009B181B18C84A94466344CA
:102370001B889B059B0D2A002932FF32D361002B5D
:102380000FD0516900290CD01400D288FEF764FDEB
:102390006369E2699446634463610021280000F0A8
:1023A0004CFB2B6850229A5A9B18B84A94466344B7
:1023B0002A002932FF321269002A67D11A88B449EB
:1023C0001140B44A0A431A8029680A88B24B1A405D
:1023D000C0239B015A40B14B13439BB20B809DE736
:1023E0000388AF4A1A40AB4B13439BB20380296862
:1023F0005023CB5A2822AA5CD2009B185B18A94A0A
:10240000944663441B889B059B0D6B64EA6B944662
:102410006344EB630021280000F01CFB2423EB5CE9
:10242000002B00D17AE72B6C002B00D076E724221A
:10243000AB5C802149420B43DBB2CC31286843526C
:102440000023AB546AE75023C35A94225200AA5C7B
:10245000D2009B181B188D4A944663441B889B0529
:102460009B0D2A002932FF32D3618C218900691823
:10247000D288FEF7F1FC2A68138883490B4080213B
:102480000B431380280000F0CDFA47E73E2A06D818
:102490005108D20700D501318902198094E751090A
:1024A000D20600D10139890289B27A4A11431980D2
:1024B0008AE7A300984640440688B6B233B2002BA0
:1024C00030DB330600D429E72B6843441A001B880D
:1024D000734919406F4B0B439BB2138028685023FC
:1024E000C35A610169180A0028321278D2009B1879
:1024F0001B186C4A944663441A889205920DA31CDB
:102500005B01E8184260C86B84466244CA635B5949
:10251000002B00D0ACE00C0028342178280000F01B
:1025200099FAFBE60388584A13408022134303803C
:102530006301EB183533FF331B78002B1ED128685D
:102540005033C35A6201AA182932FF321278D200DE
:102550009B181B184D4A944663441F88BF05BF0D46
:1025600033D06301EB181A002F32FF3212883D334B
:10257000FF3319683B00FEF76FFC26E02868630113
:10258000EB182933FF331B789A0082181288520403
:102590004BD55022825ADB00D3181B18414A94466F
:1025A00063441F88BF05BF0D32D16301EB18293387
:1025B000FF331A7892002B689C46624413883A498C
:1025C00019403A4B0B439BB21380390020000A306C
:1025D00040012A185368DB1953606301EB183D333F
:1025E000FF331A68944667441F604359002B06D096
:1025F0006201AA183932FF32126891422ED2630169
:10260000EB182933FF331978280000F016FA58E741
:102610006301EB181A003132FF3212883D33FF3369
:1026200019683B00FEF718FCBFE75022825ADB0016
:10263000D3181B18154A944663441F88BF05BF0D65
:10264000B3D06301EB181A003332FF3212883D33E6
:10265000FF3319683B00FEF7FFFBA6E76201AA18EB
:102660002932FF3211783A002800FFF70DFE28E7E3
:1026700064012C19283421782800FFF72BFE4DE641
:10268000002004BC9046F0BD8F0F0000060400003F
:10269000FF83FFFF0080FFFF8FBFFFFF8080FFFFF2
:1026A0000F8FFFFF020400008F8FFFFFC080FFFF2E
:1026B00070B504000068FEF749FA030400D57BE01A
:1026C0002068FEF743FA430500D579E02068FEF75D
:1026D0003DFA430405D5216844228B5A58480340EB
:1026E0008B522068FEF732FA830405D52168442214
:1026F0008B5A544803408B522068FEF727FAC304D4
:1027000018D521684023CA5A04208243CA5221683E
:10271000CA5A04308243CA5298239B00E35C012BBF
:102720005CD0200000F0C6F9216844228B5A46484C
:1027300003408B522068FEF709FA030557D420683E
:10274000FEF704FA030626D5216844228B5A80201E
:1027500083438B5298239B00E35C002B62D121685A
:102760004033CA5A04200243CA522168CA5A082078
:102770000243CA5298239B000122E2545423226848
:10278000D25A9208183B134099229200A35001217B
:10279000200000F009F92068FEF7D8F9830545D438
:1027A0002068FEF7D3F9C30505D5216844228B5A6A
:1027B000264803408B5270BD2000FFF7ABFD7FE73A
:1027C000216844228B5A224803408B52200000F09B
:1027D00053F900212000FFF7D2FC77E798239B00F4
:1027E0000022E2540021200000F0DEF899E7216881
:1027F0004023CA5A08200243CA5220684421425A40
:10280000144D2A4042522168CA5A04200243CA5237
:102810002068FEF79BF9C30400D590E7200000F084
:1028200037F98CE7200000F033F9B4E7216844223F
:102830008B5A094803408B52200000F016F9AFE78D
:10284000FFBFFFFFFFDFFFFFFFEFFFFFFFFEFFFF09
:10285000FFFBFFFFFFF7FFFFFFFDFFFF70B5050068
:1028600007240C4043689C4233D84BB2002B20DB3A
:102870004B0119002931FF314118C3182A33FF33A6
:1028800000221A7001238B700C708A239B00EB5C72
:10289000012B20D08A239B000122EA542868FEF7EE
:1028A000D1F8002C0ED08A239B000022EA5400208D
:1028B00010E06301190028314118C318293301229F
:1028C0001A70DFE78C239B00E9182868FEF742F9AD
:1028D000E9E7012070BD0220FCE770B504000F237A
:1028E0000B40426893422FD84BB2002B21DB0723C9
:1028F0000B405B011A002932FF328218C3182A33B9
:10290000FF330020187000239370073319401170B3
:102910008A239B00E35C012B18D08A25AD0001239C
:10292000635511002068FEF7B3F8002363550020BB
:102930000BE007230B405B011A0028328218C318F2
:10294000293301201870DEE7012070BD0220FCE76A
:1029500010B50C060DD50724214049012831401837
:10296000002A0BD00122027303811B0C438100203B
:1029700010BD49012931FF314018F1E70273C380CE
:10298000F5E702689A239B000121C150083B002112
:10299000C1545423D15A01200143D152D15A0220AB
:1029A0000143D152002070477047000010B5094C18
:1029B00000220949200000F025FA0849200000F013
:1029C0003DFA0749200000F0C3FE200000F03FFA66
:1029D00010BDC04640040020080000204400002034
:1029E0003C00002000B583B002680C4B9A4201D035
:1029F00003B000BD0A4AD169802000040143D161BF
:102A0000D36903400193019B002201211F20FFF79E
:102A1000DBFA1F20FFF70AFBEAE7C046005C004034
:102A20000010024010B501009C239B00C058403BA1
:102A30009C46614400F028FA10BD10B503009C22AA
:102A4000920080584A019B183D33FF331A6800F00A
:102A50004FFA10BD10B503009C22920080584A0125
:102A60009B18DA6B00F080FA10BD10B59C239B0018
:102A7000C05800F012FB10BD70B505009C24A400E6
:102A80000121005900F0F4FA285900F0CEFA70BD87
:102A900010B504009C239B00C05800F0ECFAA36919
:102AA000002B04D0024A136906210B43136110BDA9
:102AB00000ED00E010B59C239B00C05800F0E6FA42
:102AC00010BD000070B504001B489C239B00C4503F
:102AD0008825AD006051194B036008234360022232
:102AE00082600023C36002618361C3610362FFF7F8
:102AF000C5FA1823002200216059FFF729FF582347
:102B0000002280216059FFF723FFC023002281218A
:102B10006059FFF71DFF88235B00002201216059E7
:102B2000FFF716FF605980235B0000228221FFF728
:102B30000FFF002070BDC04678010020005C0040FF
:102B400010B588239B00C058FFF702FB002803D074
:102B5000022803D0022010BD0020FCE70120FAE784
:102B600010B514001A0088239B00C0582300FFF7FB
:102B70001CFB002803D0022803D0022010BD002037
:102B8000FCE70120FAE710B588239B00C058FFF747
:102B900049FB002803D0022803D0022010BD0020EA
:102BA000FCE70120FAE710B588239B00C058FFF727
:102BB00055FE002803D0022803D0022010BD0020BB
:102BC000FCE70120FAE710B588239B00C058FFF707
:102BD00084FE002803D0022803D0022010BD00206C
:102BE000FCE70120FAE70A0088239B00C35849B29A
:102BF000002907DB7F21114049015B182B33FF338C
:102C0000187870477F21114049015B182A331878E2
:102C1000F7E710B588239B00C058FFF7B0FA0028EB
:102C200003D0022803D0022010BD0020FCE70120C1
:102C3000FAE710B58824A4000059FFF74BFB0028E1
:102C400003D0022803D0022010BD0020FCE70120A1
:102C5000FAE710B58824A4000059FFF715FB0028F7
:102C600003D0022803D0022010BD0020FCE7012081
:102C7000FAE7000012230B80004870472400002070
:102C800004230B80004870473800002010B50A006C
:102C9000002805D00549064800F0ADFC034810BDEA
:102CA0000249034800F0A7FCF8E7C046640600208C
:102CB000A838000810B50A00034C2100034800F0B2
:102CC0009AFC200010BDC04664060020943800081D
:102CD00010B50A00002805D00549064800F08BFC15
:102CE000034810BD0249034800F085FCF8E7C046E0
:102CF00064060020B438000810B50A00002805D08A
:102D00000549064800F077FC034810BD0249034816
:102D100000F071FCF8E7C04664060020783800082F
:102D200010B50A00002805D00549064800F063FCEC
:102D3000034810BD0249034800F05DFCF8E7C046B7
:102D4000640600208438000870B5002291420FD933
:102D5000084C2368865C084DEE5401332360013231
:102D600080246400A342F1D1024B00241C60EDE7F3
:102D7000002070BD28010020B0080020F0B5DE461C
:102D8000474680B585B006008B089B4603270F4059
:102D9000019727D0002005B00CBC90469B46F0BDA3
:102DA00000230093019C18E002230093FAE7032319
:102DB0000093F7E701230093F4E74346E318013358
:102DC000F35C02AAD11D0B706B005B1998000B4BD2
:102DD000C01800F0C6FC0134A4B26B461B88A342A5
:102DE000EBD80137BB45D5D9BB009846F25C150935
:102DF0000F2313409B00024AD3589F4664080020CB
:102E0000C438000810B5002816D085239B00C3588D
:102E1000002B03D085239B000024C450002902D03E
:102E200084239B00C150FE235B000121C15402702A
:102E3000FFF748FE002010BD0220FCE7002904D067
:102E400085239B00C150002070470220FCE710B58D
:102E5000FFF776FE002010BD10B585239B00C358F8
:102E6000002B07D01B689847002801D1002010BD17
:102E70000220FCE70220FAE710B585239B00C35827
:102E80005B689847002010BD70B5040082239B004A
:102E9000C518280000F02CF9FA235B000122E2504B
:102EA000124BE25A163BE2501033E15CEA3BFF3B27
:102EB0000B40012B0FD0002B07D0022B10D07F230B
:102EC00099432000FFF76FFE03E02900200000F087
:102ED000B3FA002070BD2900200000F0D1FAF8E715
:102EE0002900200000F0EBFAF3E7C0460E020000D4
:102EF00010B504001300002929D1FA22520082588B
:102F0000032A01D0002010BD421DFF329168D26813
:102F100091420FD885239B00C3581B69002B05D015
:102F2000FE225200825C032A00D19847200000F064
:102F30009EFBE7E7891A0530FF3081608A4200D99D
:102F40000A0092B21900200000F089FBDAE785231D
:102F50009B00C3589B69002BD4D0FE225200825C98
:102F6000032ACFD19847CDE770B50400130000299C
:102F70004ED1FA2252008258022A06D080239B00AA
:102F8000E35C012B3FD0002070BDC269056AAA42F4
:102F90001ED8866929003000FDF73CF9002906D1CA
:102FA000B54204D8FC235B00E3589E421DD3852321
:102FB0009B00E358DB68002B06D0FE225200A25C87
:102FC000032A01D120009847200000F05CFBD5E7E0
:102FD000521BC26192B2190000F039FB002300229B
:102FE00000212000FFF735FEC8E70022200000F096
:102FF0002EFBFC235B000022E25000230021200076
:10300000FFF727FEBAE780239B000022E254BAE7CD
:1030100085239B00C3585B69002BB4D0FE2252006D
:10302000825C032AAFD19847ADE770B50400402316
:1030300000220021FFF794FD402588235B00E55026
:10304000D03B002280212000FFF78AFD2562FE236D
:103050005B000122E2541C33E358002B06D0852389
:103060009B00E3585B68217920009847002070BDE1
:10307000017400207047FE235B00C15CFE22FF321A
:103080008154FA3AFF3AC25400207047FE23FF33BE
:10309000C25C013BC2540020704710B5FE235B00A8
:1030A000C35C032B01D0002010BD85239B00C358B7
:1030B000DB69002BF7D09847F5E70300002002E01A
:1030C0000130C0B201331A78002AF9D1704710B527
:1030D00004004B88012B0AD181239B000122C2509E
:1030E0001033C3589B689847200000F0C0FA10BD09
:1030F0000B7803704B7843708B78CA7812029B1858
:1031000043800B794A7912029B1883808B79CA79A4
:1031100012029B18C380704710B504008021FFF78E
:1031200042FD00212000FFF73EFD10BD30B583B009
:1031300004000D004A88130A072B00D98EE09B007B
:103140004F49CB589F4684239B00C3581B68007C83
:103150006A46911D98476B4606331B88002B03D0A7
:10316000EA88002A00D07EE003B030BD037C002B4B
:1031700009D185239B00C3589B6A6A46901D9847D6
:1031800002234370E7E785239B00C358DB6A6A4646
:10319000901D984702234370DDE7D2B2052A39D843
:1031A0009200384B9B589F4684239B00C3585B6812
:1031B000007C6A46911D9847CDE784239B00C35845
:1031C0009B68007C6A46911D9847C4E784239B0056
:1031D000C358DB68007C6A46911D9847BBE784238F
:1031E0009B00C3581B69007C6A46911D9847B2E753
:1031F00084239B00C3585B69007C6A46911D9847F5
:10320000A9E784239B00C3589B69007C6A46911DF3
:103210009847A0E72900FFF77FFFA5E7037C002B75
:1032200007D185239B00C3585B6B6A46901D984766
:1032300091E72900FFF770FF96E7037C002B09D187
:1032400085239B00C3581B6B6A46901D9847072334
:10325000437080E72900FFF75FFF85E72900200022
:10326000FFF75AFF80E7191C934200D9111C8AB25C
:103270006B46D9800100200000F0DBF974E7C046FE
:10328000043900082439000870B504008B88002B2D
:1032900022D1CB88002B1FD18B787F251D40FE23A8
:1032A0005B00C35C032B0FD0FF235B00C5542900D8
:1032B000FFF7AFFC200000F0DAF9002D07D0FE2365
:1032C0005B000222E2540AE0FFF726FF07E0FE233C
:1032D0005B000122E25402E02000FFF71DFF70BDF9
:1032E00070B504000D008978284B197001290AD89F
:1032F000FE235B00C35C022B09D0032B1ED02900E8
:10330000FFF70AFF02E02900FFF706FF70BD002962
:1033100011D04160FE235B000322C254FFF79CFDE5
:10332000022803D0200000F0A2F9EFE729002000D6
:10333000FFF7F2FEEAE700F09AF9E7E7002911D07B
:10334000436899421ED0D9B2FFF796FD0F4B19780A
:1033500061602000FFF780FD02280ED0200000F001
:1033600086F9D3E7FE235B000222C2544160FFF7D7
:1033700083FD200000F07BF9C8E729002000FFF75B
:10338000CBFEC3E700F073F9C0E7C046240100207C
:1033900010B5CB88012B09D1FE235B00C35C022B47
:1033A00007D0032B0DD0FFF7B7FE01E0FFF7B4FE07
:1033B00010BD0023836001000831012200F039F9BB
:1033C000F6E7011D012200F034F9F1E710B5FE2304
:1033D0005B00C35C023BDBB2012B0ED80123C36050
:1033E00081239B00C358002B01D00323C36001003D
:1033F0000C31022200F01DF910BDFFF78DFEFBE736
:1034000010B50400FE235B00C35C023BDBB2012B62
:103410000ED84B88012B0AD181239B000022C25079
:103420001033C3589B689847200000F020F910BD66
:10343000FFF772FEFBE7000010B54B78092B19D897
:103440009B000E4AD3589F46FFF770FE002010BD28
:10345000FFF71AFFFAE7FFF743FFF7E7FFF798FFD9
:10346000F4E7FFF7B3FFF1E7FFF731FEEEE7FFF711
:10347000C7FFEBE7FFF750FEE8E7C0463C3900081E
:1034800070B504000D00FE235B00C35C032B13D159
:103490000B79012B0DD885239B00C3589B68984757
:1034A000EB88002B01D0002070BD200000F0DFF879
:1034B000F9E7FFF731FEF6E7FFF72EFEF3E770B509
:1034C00005000C008A88D1B2207860230340202BAD
:1034D00008D1F533FF33EB589B682100280098474B
:1034E000002070BD6378012B2CD0002B52D0032B11
:1034F000F6D1FA33FF33EB5C022B06D0032B0CD052
:1035000021002800FFF708FEEAE70029E8D080291B
:10351000E6D02800FFF747FBE2E76388002B06D1DF
:10352000002904D0802902D02800FFF73CFB852326
:103530009B00EB589B68210028009847280000F06A
:1035400096F8CDE7FE235B00EB5C022B06D0032B45
:103550000CD021002800FFF7DFFDC1E70029BFD014
:103560008029BDD02800FFF71EFBB9E76388002B38
:10357000B6D14B0603D1280000F079F8B0E7280057
:10358000FFF721FB85239B00EB589B682100280057
:103590009847F0E7FE235B00EB5C022B06D0032B81
:1035A0000AD021002800FFF7B7FD99E74B0697D016
:1035B0002800FFF7F8FA93E7130612D47F240C4093
:1035C000103424012C1904342800FFF70CFB0028C8
:1035D0000ED00123236002222100280000F029F8E8
:1035E0007EE77F240C40013424012C190434EBE7DE
:1035F00000232360EFE770B504000D0016000028DB
:1036000016D0FFF75AFD0130400080B2308028709C
:1036100003236B70013B08E001345A1CD2B2E95419
:103620000233DBB2AA180021117021780029F3D1EE
:1036300070BD10B51300FA22520002248450836139
:10364000C3610A000021FFF7F4FA002010BD10B595
:1036500013000A000021FFF7ECFA002010BD10B59E
:1036600013000A000021FFF7F4FA002010BD10B586
:10367000FA235B000422C250002300220021FFF73E
:10368000D8FA002010BD10B5FA235B000522C25005
:10369000002300220021FFF7DCFA002010BD00000B
:1036A000044B1B78012B01D000207047014B0022F6
:1036B0001A70F9E72C010020852303800048704729
:1036C0007C00002070B5040087239B00C25804339F
:1036D000C3580A314901591889881368054D2800D3
:1036E000984740232A0001212000FFF7B2FA00206A
:1036F00070BDC0467008002010B50400054B0022C4
:103700001A608121FFF73FFA01212000FFF73BFA01
:10371000002010BD3001002010B504000A4B1860D5
:10372000402302228121FFF71BFA402302220121BC
:103730002000FFF715FA4023044A01212000FFF77B
:1037400088FA002010BDC04630010020700800201B
:10375000002904D087239B00C1500020704702201D
:10376000FCE710B50288541C8388013B2340448841
:10377000A3420CD00B7881688B54038801339BB231
:103780008288013A12B213400380012010BD00204C
:10379000FCE770470D4885460D480E490E4A002348
:1037A00002E0D458C4500433C4188C42F9D30B4AF5
:1037B0000B4C002301E013600432A242FBD3FFF75D
:1037C000E8FF00F011F8FCF703FEFEE700400020E0
:1037D00000000020080100207C39000808010020BA
:1037E000B0090020FEE7000070B500260C4D0D4C1E
:1037F000641BA410A64209D1002600F021F80A4D4E
:103800000A4C641BA410A64205D170BDB300EB584E
:1038100098470136EEE7B300EB5898470136F2E7D8
:1038200074390008743900087439000878390008C0
:1038300003001218934200D1704719700133F9E761
:10384000F8B5C046F8BC08BC9E467047F8B5C046FF
:08385000F8BC08BC9E4670475D
:1038580002030405060708090A0B0C0D0E0F1010C9
:103868000102030405060708090A0B0C0D0E0F10C8
:103878004D49444920436F6E666967004D49444984
:1038880020496E7465726661636500004F747465E3
:103898007220536369656E7469666963000000008D
:1038A8004D494449204469616C7300003030303020
:1038B800303030303030314100000000A02D000899
:1038C800A02D0008A82D0008AE2D0008AE2D000878
:1038D800B42D0008A82D0008AE2D0008AE2D000854
:1038E800AE2D0008AE2D0008AE2D0008A82D00084A
:1038F800A82D0008AE2D0008B42D00085C32000881
:10390800463100086C3100089A3100085C32000822
:103918005C3200081C3200083A320008A83100085E
:10392800BA310008CC310008DE310008F031000857
:1039380002320008623400086E340008743400084B
:10394800683400087434000850340008483400080B
:10395800743400085C340008563400080000000085
:0C3968000000000001020304060708092B
:04397400E90000085E
:04397800C100000882
:10397C000100000004000000752C0008812C0008D8
:10398C00B52C00088D2C0008D12C0008F92C00084F
:10399C00212D000812010002020200400912010050
:1039AC000002010203010000040311047D2D000834
:1039BC00492D000819370008F936000800000000EE
:1039CC000000000000000000A1360008C536000809
:1039DC0000000000000000000000000000000000DB
:1039EC00B936000800000000000000000902850044
:1039FC00020100800A0904000000010100000924F2
:103A0C000100010900010109040100020103000089
:103A1C0007240100014300062402010100062402D0
:103A2C0002020006240201110006240202120009FF
:103A3C002403010301020100092403020401010112
:103A4C0000092403011301120100092403021401CB
:103A5C0011010009050102400000000006250102C9
:103A6C000111090581024000000000062501020336
:083A7C001300000000127A00A3
:040000050800379523
:00000001FF
